:10740000E0E0F0E0859194910196089520E82093C2
:1074100061001092610081E085BF82E085BF87E056
:1074200084B981E785B917B8469A10BA80EC81BB58
:1074300084EA8BB984EF8AB980E58CBD81E08DBD8B
:10744000089580EE8BB98BEA55D0109289008AEFAF
:107450008093880082E080936F0083E080938100B6
:10746000E7E0F1E05CD0E331E9F7A5E2B4E0E3E185
:10747000F1E003E010E101900D921A95E1F7A059B7
:10748000BF4F0A95B9F753D081E08093D7008AE4C3
:1074900082BF1092D8001092E2001092DA0010928F
:1074A000E10080E808D019BC1EBA1092E00072D446
:1074B00089E05ED481E98093D8000895F201F999BA
:1074C000FECFF2BDE1BD0895F9DFF89A80B508C09E
:1074D000F5DF1FBA80BD0FB6F894FA9AF99A0FBE7D
:1074E00031962F01089590E81BD08D939A95E1F77E
:1074F000089586E008D010C083E005D08F2F10D00B
:107500008E2F0ED080E05F9A5A980AC005D085E091
:10751000FADF06D080FDFDCF5A9A5F9808958191D9
:107520008EBD8DB5000087FFFCCF8EB50895EDEEC2
:10753000F2E090EB5C98892FF3DF80E1F1DF5C9A59
:10754000EEDF8DEE8E278F77D9F79395983B91F7E5
:107550000895EBEDF1E08191908101969083829303
:10756000092E0AF400940091D90106FB5EF0009602
:10757000929111F493959083000C081620F4289AA8
:10758000289A289A0895937009F42898913009F45C
:107590002898923009F428980895E2EDF1E0978157
:1075A0009923FAF083B180958077369B84607F9B26
:1075B00082607E9B81609581891310C0968199239A
:1075C00081F49381891306C09481992396E959F037
:1075D00080E00AC083839095892304C085839AE064
:1075E000968380E09FEF9483828308958091D901F0
:1075F00086FFC5DF22243324E2EDF1E010861186F8
:107600001286EDEEF1E08091D40184FD1BC086FD71
:1076100032C080FF0895C685CC23E1F3F894289802
:107620000088F785E02D68DFE0E0F0E0ADEEB1E046
:107630005ADFADEEB1E042D3E058FF4FCA95B1F743
:107640006BDFC9C18301282D6090F6017090F501B0
:1076500046D019F48823C1F70895380188243FD013
:10766000E1F58091F401821709F483016090F8013B
:107670007090F701F4CF6090F8017090F7012FD06F
:1076800081F48823C1F708959FEF85FD08C082FD2E
:1076900005C081FF0895B4DEE9F39DC191E097FB39
:1076A000890E662477248301222719D0B1F4882318
:1076B00089F38091F40136F0881650F4821730F087
:1076C000213003C0881520F4281710F48301282FD7
:1076D0006090F8017090F701E8CF3801822EF30135
:1076E0000BDFADEEB1E0FFDECDEED1E0E0E0F1E0AA
:1076F00097E009908191081621F49A95D1F70880B6
:1077000080100ACFC9E0EFDECA95E9F705DF0FDF89
:047710008827089529
:1077140041524455424F59D5F08D14A1C881CFD957
:10772400F1AF000000FFFFCFCFFFFFFFFFCFCFFF80
:10773400FF0000FE067E7E06FE46565616FE0656E0
:10774400461EFE3F61E9E3FFE3EBE3FFE3EBE3FF08
:10775400E16B3F12011001020000084123360001D1
:10776400000201000109023E000201008032090406
:107774000000010202010005240010010424020497
:107784000524060001070582030800FF090401001F
:10779400020A000000070504021000010705830225
:1077A40010000104030904220341007200640075FF
:1077B4000069006E006F0020004C0065006F006ED1
:1077C400006100720064006F0018034100720064DD
:1077D40000750069006E006F0020004C004C0043EF
:0277E4000000A3
:1078000011241FBE8DEF9AE09EBF8DBF04B714BE3A
:1078100088E18093600010926000409100085091D0
:1078200001086F917F91A6C00F928F939F931F9233
:107830000FB60F9211244F936F938091DA0080FF5F
:107840004CC038C00F920FB68F939F93EF93FF9366
:1078500088278093850080938400E2EDF1E0978192
:10786000907261F490818917980B908309F45D9A66
:1078700091818917980B918309F4289A96819150E8
:1078800008F096839481915008F09483881639F417
:107890001E9B05C0B5DD19F0C10101961C01FF91C9
:1078A000EF915CC080E189BD82E189BD09B400FE31
:1078B000FDCF08958091D80080FF0FC08091DA003D
:1078C0008E7F8093DA008091D90080FF04C0EADFC8
:1078D00081E08EBB02C019BC1EBA8091E10080FF1E
:1078E0000BC040D280FF08C040D28091D800806297
:1078F000E2DD19BC85E08EBB8091E10084FF1AC0F7
:1079000031D284FF17C0CEDF8091D8008F7DD3DDC8
:107910008FEE2AD027D28F7E81602AD28091DD011E
:10792000882331F48091E30087FD02C081E001C02B
:1079300084E08EBB8091E10083FF0CC013D283FFF3
:1079400009C087EF11D082E08EBB1092DD010BD011
:107950000CD220D26F914F910F901F909F918F91D9
:107960000FBE0F9018958EEF0090E1000822009254
:10797000E10008954BDDA0E0B1E0E4E1F7E7059018
:107980000D92A13DE1F71D92BB30E9F701FD0FC05B
:1079900000FF03C01E9B0BC008C003FF08C0675751
:1079A000774729F04757574711F02ADDA1F449DD01
:1079B000222433243101882492DE789447D00ED3D8
:1079C000ECDD62DE811411F011DEF8CFC2DDC10101
:1079D000805B964398F3F89489EB8CDD81E080938B
:1079E000E00010926F0010928100109285001092BA
:1079F000840081E085BF15BEC2DD5D9A289A0C9493
:107A00000000ABD107C058D102C0E5D239F0A7D1F0
:107A100082FFFBCF85FFF7CF8091F1000895082EFC
:107A200083E09CD185FD07C091D102C0D4D269F01A
:107A300096D180FFFBCF0092F1008091D90185FBA8
:107A400026F05D9884E68093D201089586D182FF66
:107A50004EC18091D90185FB26F0289884E6809359
:107A6000D301CFDF182F853431F48CEB94E31C0164
:107A700025DD8DE00CC1843511F4C3DFFACF8C34E1
:107A8000C1F38035B1F3843721F484E4C8DF80E0AA
:107A9000FEC0813611F489E5FAC0813429F4B1DFE2
:107AA000582EAFDF482EE5CF803711F483E5EFC0C5
:107AB000833539F4C0E0D1E08991B1DFC730E1F717
:107AC000E7C0863521F481E3AADF84E3E0C086378E
:107AD00081F481E37F9B8E5F7E9B8F5FA0DF81E4DB
:107AE0001C9B885F369B8C5F1D9B8E5F1E9B8F5FF0
:107AF000CEC08837A9F485DF8093D901289A84FD08
:107B000028985D9A83FD5D98289A81FD2898289A87
:107B100082FD2898289A80FD289887FD8824A9CF7F
:107B20008A3649F48FE9EFDCC3E0FADC78DFCA95E6
:107B3000E1F7F2DCADC0833731F487E870DF85E927
:107B40006EDF8EE1A4C0853639F4E0E8F3E7C7D0F4
:107B5000E058F040E0F78DCF823631F489E55FDF01
:107B600080E05DDF80E893C0823419F0873609F049
:107B70007AC02224332445DFD82F43DFC82F41DFCA
:107B8000082F8354843008F081C0063411F4440C6B
:107B9000551CF20110926F001736A1F4033471F4F2
:107BA00083E0ABDCBDDC3BDF2197E1F7B5DC08C04F
:107BB000063411F4859101C087DC31DF2197C2F7CB
:107BC0002F0149C00334A1F48E2F8F7021F491DC72
:107BD00080E293DC9BDC8DDC82E08FDC12DFA0DCBA
:107BE000CA95E1F793DC3196DA9571F72F0131C030
:107BF0000634F1F49F01F437D8F471D019C001DFD5
:107C0000063461F4C0FB46F0F43728F4182E81E006
:107C100087BFE89511243296082E0AC0043439F43F
:107C2000DF01B370A351BD4F8D93319601C050DC7D
:107C300021972AF7043431F42F01F370FE2B49F415
:107C400076DC07C0063429F42F01F901F43708F473
:107C500044D08DE0E4DE063411F45694479482E07B
:107C600080936F0015C08237E1E049F08634E0E090
:107C700031F08E34E3E019F0813531F4E2E0F0E0E8
:107C800089E087BF849103C08B3111F08FE3C7DE99
:107C900083E0B1D15BD095FF03C009C09CD139F11D
:107CA0005ED080FFFBCF52D002C095D101F157D0FA
:107CB00080FFFBCF84E09FD18BE749C0F437B8F455
:107CC0000ED090E40D901D9081E087BFE89532962C
:107CD0009A95C1F71124E058F04085E001C083E097
:107CE00001D081E187BFE89507B600FCFDCF08957C
:107CF0009091E5018091E601913231F0913A61F580
:107D0000813251F538D087C0803231F534D063D11B
:107D1000E9F08530D9F023D083FD18C082FFF7CF7A
:107D200004C07ADE8193615031F09091F30080912C
:107D3000F200892BB1F7C0DF611549F704C04BD1C0
:107D400029F0853019F00BD080FFF9CF8EE79091A4
:107D5000E80089238093E800089584E04CD1809165
:107D6000E80008958091E2000895FCDF8E7F806135
:107D70008093E20008952DD1EEEDF1E067E00895E3
:107D800082E061EC09D083E061E802D084E060E841
:107D900042E103C080E060E042E02DD181E007D005
:107DA0001092ED006093EC004093ED0008959091E7
:107DB000EB00892B8093EB00089560E0923039F05E
:107DC000933041F0913099F4E3E462E110C0E5E5CD
:107DD0006EE30DC0813018F4E3E964E008C019F4E3
:107DE000E7E962E204C0823011F4E9EB68E1F1E016
:107DF00008958091E50188234CF402C0ECD051F045
:107E0000AEDF82FFFBCF58CFE6D021F0A8DF80FFA6
:107E1000FBCF9CDF08954091EB015091EC01461798
:107E2000510510F490E028C0611511F0462FFACFEB
:107E30008DDF40E0F7CFCFD059F1853049F18FDFAA
:107E400083FD3ACF8CDF82FD20C080FF15C03091CA
:107E5000F3002091F20005C081918093F100415020
:107E60002F5F411519F028303105B0F350E028306C
:107E7000310509F451E06ADF4115E9F65523D9F6D9
:107E800004C0A9D029F0853019F069DF82FFF9CF4D
:107E900013CFE5EEF1E0C0DD8193ED3EE1F728DFA1
:107EA0005EDF83FF91C08091E5019091E601913002
:107EB00009F170F09330F1F0953009F444C0963038
:107EC00009F456C0983009F460C0993059F767C07A
:107ED000823841F78091E9018DD02091EB0010921A
:107EE000E90077D02295269521702093F100109219
:107EF000F10052C0882311F08230A1F68F718230D8
:107F000089F68091E7018823D1F42091E901277057
:107F100049F22093E9008091EB0080FF10C093307C
:107F200011F480E20BC080E142DF81E0880F2A95E6
:107F3000E9F78093EA001092EA0088E038DF1092B7
:107F4000E90047D02AC0882391F41091E701106816
:107F50000FB7F8943ED04DDF02DF80FFFDCF1093C6
:107F6000E300103883E009F482E08EBB0FBF2CC021
:107F70008058823048F58091E7019091E8011DDF3B
:107F8000603011F126D047DF1FC08038E9F421D0DE
:107F90008091DD018093F100D9DE2BDF15C08823AD
:107FA00099F49091E701923078F49093DD0111D02B
:107FB00020DF8091DD01882321F48091E30091E0AE
:107FC00087FD94E09EBBDCDECADE83FF089580E27D
:107FD000EEDE87EFBCCE8EB388230895FCDF69F018
:107FE0008091E9008F931092E900B9DE83FF01C010
:0C7FF00050DF8F9187708093E9000895A6
:047FFC005FCEFBDC7D
:040000030000740085
:00000001FF
